:100000000C9463000C94C4070C94F1070C948B00BF
:100010000C948B000C948B000C948B000C948B0034
:100020000C948B000C948B000C948B000C948B0024
:100030000C948B000C948B000C948B000C948B0014
:100040000C941E080C948B000C94FE0A0C94300B3C
:100050000C948B000C948B000C948B000C948B00F4
:100060000C948B000C948B0000000008000201002F
:100070000003040700000000000000000102040863
:100080001020408001020408102001020408102002
:10009000040404040404040402020202020203032E
:1000A00003030303000000002300260029000000D2
:1000B0000000250028002B0000000000240027007D
:1000C0002A000F02600B11241FBECFEFD8E0DEBF65
:1000D000CDBF11E0A0E0B1E0ECEEF9E102C0059087
:1000E0000D92AC3CB107D9F724E0ACECB1E001C013
:1000F0001D92AF38B207E1F710E0C6ECD0E004C0C3
:100100002297FE010E94DC0CC23CD107C9F70E9475
:10011000A40B0C94F40C0C940000F8941092E101E0
:100120001092E0018091DE019091DF01009721F0B3
:100130009093DD018093DC011092DF011092DE01CB
:1001400078940895F8946091DC017091DD0100903D
:10015000E00102C0769567950A94E2F7617084E049
:100160000E945A098FE090E00E94B30885E00E9447
:1001700090092091DC013091DD01892B81F081E033
:1001800090E0A0E0B0E00090E00104C0880F991F6B
:10019000AA1FBB1F0A94D2F7822B932B11C081E0B8
:1001A00090E0A0E0B0E00090E00104C0880F991F4B
:1001B000AA1FBB1F0A94D2F78095909582239323A0
:1001C0009093DD018093DC018091E0019091E10149
:1001D000019660E170E00E94A40C9093E10180938D
:1001E000E001789408950F931F93CF93DF938CECE5
:1001F00091E00E947B07882309F4A8C08CEC91E071
:100200000E949A07882309F4A1C061E271E082EF9D
:1002100093E00E94F10B4AE050E06091CC0182EF44
:1002200093E00E94860C82EF93E00E94FA0B6CE24E
:1002300071E082EF93E00E94F10B10E08091CC011D
:100240001817C8F4C12FD0E0C453DE4F8981803124
:1002500018F460E071E002C06FE171E082EF93E0BA
:100260000E94F10B40E150E0698182EF93E00E942F
:10027000860C1F5FE3CF82EF93E00E94FA0B10928F
:10028000DB011092DA01C0E02091CC018091DA010B
:100290009091DB01C21768F4EC2FF0E0E453FE4FBD
:1002A00061810E9415029093DB018093DA01CF5F98
:1002B000EBCF90689093DF018093DE0163E071E003
:1002C00082EF93E00E94F10B6091DE017091DF01FB
:1002D00040E150E082EF93E00E948D0C62E171E01A
:1002E00082EF93E00E94F10B00E110E0C0E0D0E863
:1002F0008091DE019091DF018C239D23892B11F0E9
:1003000061E301C060E382EF93E00E94F30BC03130
:10031000D10541F0C11581E0D80721F0C11580E178
:10032000D80731F46FE171E082EF93E00E94F10BA6
:10033000D695C79501501109D9F682EF93E00E9436
:10034000FA0B64E170E080E090E004C065E070E0EA
:1003500080E090E0DF91CF911F910F910C948B087A
:10036000CF936EE68CEC91E00E942403C82F6BE3E0
:1003700071E082EF93E00E94F10B40E150E06C2FBE
:1003800082EF93E00E94860C60E271E082EF93E0DE
:100390000E940E0CC150CE3F38F068E571E082EF4C
:1003A00093E0CF910C940E0CCF91089526E040E09D
:1003B00051EE60E070E082EF93E00E949C0A0E94A0
:1003C0005E028CEC91E00E945C046BE971E082EFCC
:1003D00093E00E940E0C0E94B00162E082E00E9455
:1003E000210943E050E062EA70E080E00E94A40747
:1003F00062E083E00E94210943E050E06DE870E094
:1004000081E00E94A40760E085E00E94210961E08C
:1004100084E00E94210960E084E00C945A0949E0DC
:100420006AE08CEC91E00C94A202DF92EF92FF92D2
:100430000F931F93CF93DF93D82E70E02091E203A8
:100440003091E303232B31F5E2EEF1E040E050E0A0
:10045000EA01A8E0B0E020E030E07E01E226F326E9
:1004600036952795E0FE04C081E0282780EA3827EA
:10047000D695C795119789F7219331934F5F5F4FB9
:10048000411581E0580721F721E030E03093E30384
:100490002093E203092F10E0FB01ED25EE0FFF1F73
:1004A000EE51FE4F8081918180279127DF91CF917E
:1004B0001F910F91FF90EF90DF900895CF93CFB7EA
:1004C000F8948091E403811127C0EAE9F0E0849177
:1004D000E6E8F0E09491E82FF0E0EE0FFF1FE8541B
:1004E000FF4FA591B4918C91892321F461E08AE0BA
:1004F0000E945A0961E08AE00E9421098CB580615E
:100500008CBD8CB580648CBD61E08DE00E942109BA
:1005100061E08BE00E9421098091E4038F5F80936A
:10052000E403CFBFCF9108958EBD00000DB407FE48
:10053000FDCF8EB508958CB58F7D8CBD8CB5837F36
:100540008CBD08950F931F93CF93DF931F92CDB768
:10055000DEB78C01862FF801648761E049830E9431
:10056000210961E0F80184850E945A094981F80156
:10057000458761E0842F0E94210960E0F8018585AC
:100580000E945A09C8010F90DF91CF911F910F91DE
:100590000C949B02EF92FF921F93CF93DF931F92D5
:1005A000CDB7DEB77C01162F60E0FC01848549835E
:1005B0000E945A09812F8E770E9494024981842FCC
:1005C0000E94940261E0F70184850F90DF91CF9142
:1005D0001F91FF90EF900C945A09CF92DF92EF9207
:1005E000FF920F931F93CF93DF9300D0CDB7DEB769
:1005F0008C01E62EF42E60E0FC01848529833A8389
:100600000E945A098E2D8E770E9494022981E22E33
:10061000C22E3A81D32E8C2D8E198F1530F4F6010F
:1006200081916F010E949402F6CF61E0F801848508
:100630000F900F90DF91CF911F910F91FF90EF904E
:10064000DF90CF900C945A091F93CF93DF93EC0166
:10065000162F60E08C850E945A09812F8E77806862
:100660000E94940280E00E949402182F61E08C8521
:100670000E945A09812FDF91CF911F9108957F9297
:100680008F929F92AF92BF92CF92DF92EF92FF92A2
:100690000F931F93CF93DF936C01842EE9014423C2
:1006A00009F453C0162F1E77106860E0FC018485A2
:1006B0000E945A098A94812F0E9494027C2EEC2E6B
:1006C000FD2EAA24A394B12C8E2D8719881528F508
:1006D00081111AC00023C1F0802F912C883048F47A
:1006E0009501082E01C0220F0A94EAF7922A8F5F23
:1006F000F5CF812F0E949402992D90952881922305
:100700008921982B988305C0812F0E949402F701BC
:100710008083FFEFEF1AFF0AD7CFC80DD11D80E00D
:100720000E949402888361E0F6018485DF91CF9175
:100730001F910F91FF90EF90DF90CF90BF90AF90FF
:100740009F908F907F900C945A09DF91CF911F91C9
:100750000F91FF90EF90DF90CF90BF90AF909F9060
:100760008F907F900895EF92FF921F93CF93DF9326
:100770001F92CDB7DEB77C01162F49830E94240358
:100780004981482B612FC7010F90DF91CF911F91B5
:10079000FF90EF900C94CA02EF92FF921F93CF93B9
:1007A000DF931F92CDB7DEB77C01162F49830E94DD
:1007B0002403498140954823612FC7010F90DF91A1
:1007C000CF911F91FF90EF900C94CA02DF92EF92AD
:1007D000FF920F931F93CF93DF93EC018B01D42EE5
:1007E000790140E062E00E94CA0244E06AE0CE0182
:1007F0000E94CA0240E864E1CE010E94B30398015E
:100800004D2D62E1CE010E94ED0243E062E0CE0197
:100810000E94CA0208E813E16AE0CE010E942403A4
:1008200082FD05C001501109B9F784E012C040E013
:1008300062E0CE010E94CA0264E4CE010E94240359
:10084000F701808362E4CE010E942403F7018183D3
:1008500081E0DF91CF911F910F91FF90EF90DF909A
:100860000895CF93DF93EC014FE062E00E94CA024B
:1008700062E370E080E090E00E948B0862E0CE01CD
:100880000E94240384FDFACFDF91CF910895CF9386
:10089000DF93EC0168E20E942403982F9370933059
:1008A00041F0482F436068E2CE01DF91CF910C9474
:1008B000CA02DF91CF910895CF93DF93EC018D852C
:1008C0000E949009892B59F461E08D850E945A0994
:1008D00062E370E080E090E00E948B0803C0CE01EC
:1008E0000E94310440E864E5CE010E94CA0249EA50
:1008F00066E5CE010E94CA0243E068E5CE010E948F
:10090000CA0248EE6AE5CE010E94CA0240E46AE2E9
:10091000CE010E94CA024DE362E2CE010E94CA02E9
:10092000CE01DF91CF910C9447042F923F925F92BA
:100930006F927F928F929F92AF92BF92CF92DF92EF
:10094000EF92FF920F931F93CF93DF9300D000D0CD
:10095000CDB7DEB73C01962E542E302E082DA114B3
:10096000B10419F0F501408101C040E0242EF0E10E
:100970000F9F200C112440E062E0C3012B833C83D5
:100980000E94CA024FE768E0C3010E94CA0240E821
:1009900064E1C3010E94B3032B813C81432D62E1DA
:1009A000C3010E94ED02422D6AE1C3010E94CA0206
:1009B000492D62E0C3010E94CA028CE0981205C072
:1009C00040E86AE1C3010E94B30390ED292E97E04D
:1009D000392E68E0C3010E942403982F952139F431
:1009E00080FD62C0E1E02E1A310899F75DC06CE02D
:1009F000C3010E942403982E837109F057C0E114AB
:100A0000F104F1F0C114D104D9F064E1C3010E94F2
:100A10002403482FF6018081841708F449C04083DD
:100A2000970162E1C3010E943F0368E1C3010E9494
:100A30002403182F1770A114B10411F0F5011083CD
:100A400093FC38C0E114F104B9F1C114D104A1F14F
:100A5000888D882389F1F6014081413019F41430E2
:100A600019F420C0423010F488E027C01111FCCFE7
:100A700042509E012F5F3F4FB701C3010E94E60322
:100A80008130D9F4F6018081E80EF11CF70132972C
:100A9000908189819813E8CF319690818A8198134B
:100AA000E3CF0AC089E009C084E007C082E005C046
:100AB00085E003C083E001C081E00F900F900F90AC
:100AC0000F90DF91CF911F910F91FF90EF90DF90EA
:100AD000CF90BF90AF909F908F907F906F905F90DE
:100AE0003F902F9008958F92AF92BF92CF92DF9256
:100AF000EF92FF920F931F93AF928C2C57016801D6
:100B00007901042F9B0140E36CE00E9495040F9053
:100B10001F910F91FF90EF90DF90CF90BF90AF901B
:100B20008F9008954F925F926F927F928F929F92D3
:100B3000AF92CF92EF92FF920F931F93CF93DF93D9
:100B400000D0CDB7DEB73C016A832A0149014115C7
:100B5000510531F1F9018081823010F140E86CE1FA
:100B6000C3010E94CC0387E08983A12CC12CCE0154
:100B700001967C018401920141E0BE016E5F7F4FCE
:100B8000C3010E947305813061F4F40180818230D9
:100B900011F082E006C089818111FBCF81E001C0A4
:100BA00085E00F900F90DF91CF911F910F91FF90F3
:100BB000EF90CF90AF909F908F907F906F905F90CD
:100BC0004F9008959A01AB0166E20C9492052F9222
:100BD0003F924F925F926F927F928F929F92AF92CD
:100BE000BF92CF92DF92EF92FF920F931F93CF931A
:100BF000DF93CDB7DEB72D970FB6F894DEBF0FBEEB
:100C0000CDBF3C012B01342E20E5241708F40BC185
:100C100040E86CE10E94CC03BB24B39432E0B316ED
:100C200091F043E0B416E1F081E0B81200C183E92D
:100C300089833320D1F041E0D2018C91853008F4D2
:100C400040E0D12C17C085E98983332081F041E051
:100C5000F2018081883008F440E073E0D72E0AC0AA
:100C600087E9898366E0D62E04C0D12C02C053E008
:100C7000D52E40E0532DF8EFDF9E500D112457FD87
:100C800050E0442321F088E88B8373E001C072E0D8
:100C900091E0852F877009F490E0852F85958595E3
:100CA0008595890F21F4442311F1585F20C0442316
:100CB00011F063E001C064E0861708F4682F80E05B
:100CC00090E092012D0D311DE72FE80FA1E0B0E07B
:100CD000AC0FBD1FAE0FB11DFD01D901A80FB91F8B
:100CE0001196AC91A0830196861770F3DCCF43E098
:100CF000242E503204F1B0E7BA838C819B8189277E
:100D00009D8189279E8189278F839E01285F3F4F80
:100D100047E0BE016F5F7F4FC3015D870E94E6031E
:100D20005D85813009F0CEC01B862A86FE0137968C
:100D30004F0179E01EC0952F97709B87252F259531
:100D40002595259582E0820F392FF0E18F9F300D98
:100D500011243A8371E0911101C070E0780F88246A
:100D60008394912C8C0E9D1E880E911C87E0821B13
:100D70008A87CB844C2D4295407F4C0D6AE1C3019C
:100D80005D877C870E94CA02A12C9E01255F3F4F90
:100D900079018E01065F1F4F94017C85472FBE01AC
:100DA0006F5F7F4FC3010E9473055D858330A1F59E
:100DB0006CE1C3010E9424035D8585FD36C0482F88
:100DC0004F7109F440E2842F90E0252F332727FD4F
:100DD0003095281739075CF5542F019787709927AC
:100DE000242F2595259525952F5F31E0811101C090
:100DF00030E0230FE1E0F0E0EC0FFD1FE20FF11D0A
:100E0000A1E0B0E002C0AA0FBB1F8A95E2F7CD01B6
:100E10009081982B90836DCF813009F053C0503270
:100E200044F450E268CF87E04DC083E04BC086E0D9
:100E300049C08B81883819F052E044E002C053E089
:100E400043E080E090E092012D0D311DF901E80FA3
:100E5000F91F652F680FA1E0B0E0AC0FBD1FA60F12
:100E6000B11D6C9161830196841780F38A8583306C
:100E700031F58B85811123C09E012D5F3F4F41E0ED
:100E8000B401C3010E94E6038130E1F49B81F401C7
:100E90008181981316C09C818281981312C0808131
:100EA00082FF02C0B394BACED2011B968C931B97DB
:100EB0008B2D880F8B0D8F5F8C9381E003C082E0B8
:100EC00001C088E02D960FB6F894DEBF0FBECDBFEF
:100ED000DF91CF911F910F91FF90EF90DF90CF9016
:100EE000BF90AF909F908F907F906F905F904F904A
:100EF0003F902F900895CF93DF9300D01F92CDB7EE
:100F0000DEB722E02B83AE014D5F5F4FBE016F5F06
:100F10007F4F0E94E205813031F091E0833009F08B
:100F200090E0892F01C081E00F900F900F90DF912A
:100F3000CF91089540E0BC010E94E70591E0813027
:100F400009F090E0892F08958230E8F4E82FF0E06E
:100F5000EE0FFF1FEB51FC4F71836083813041F036
:100F6000809169008C7F842B80936900E89A0895B2
:100F700080916900440F551F440F551F837F842BB8
:100F800080936900E99A08951F920F920FB60F920D
:100F900011242F933F934F935F936F937F938F937E
:100FA0009F93AF93BF93EF93FF938091E50390914D
:100FB000E603892B29F0E091E503F091E60309951A
:100FC000FF91EF91BF91AF919F918F917F916F9121
:100FD0005F914F913F912F910F900FBE0F901F90F7
:100FE00018951F920F920FB60F9211242F933F93D3
:100FF0004F935F936F937F938F939F93AF93BF9321
:10100000EF93FF938091E7039091E803892B29F0F8
:10101000E091E703F091E8030995FF91EF91BF910B
:10102000AF919F918F917F916F915F914F913F9180
:101030002F910F900FBE0F901F9018951F920F9237
:101040000FB60F9211242F933F938F939F93AF93DB
:10105000BF938091EA039091EB03A091EC03B091D0
:10106000ED033091E90323E0230F2D3720F401969F
:10107000A11DB11D05C026E8230F0296A11DB11DBB
:101080002093E9038093EA039093EB03A093EC038E
:10109000B093ED038091EE039091EF03A091F003E4
:1010A000B091F1030196A11DB11D8093EE039093C1
:1010B000EF03A093F003B093F103BF91AF919F9121
:1010C0008F913F912F910F900FBE0F901F90189509
:1010D0003FB7F8948091EE039091EF03A091F00355
:1010E000B091F10326B5A89B05C02F3F19F00196DA
:1010F000A11DB11D3FBF6627782F892F9A2F620F40
:10110000711D811D911D42E0660F771F881F991F79
:101110004A95D1F70895CF92DF92EF92FF92CF9345
:10112000DF936B017C010E946808EB01C114D104BC
:10113000E104F10489F00E94A30C0E9468086C1B72
:101140007D0B683E734090F381E0C81AD108E10836
:10115000F108C851DC4FEACFDF91CF91FF90EF90BB
:10116000DF90CF900895019739F0880F991F880F6D
:10117000991F02970197F1F70895789484B58260DA
:1011800084BD84B5816084BD85B5826085BD85B52B
:10119000816085BDEEE6F0E0808181608083E1E8DA
:1011A000F0E0108280818260808380818160808312
:1011B000E0E8F0E0808181608083E1EBF0E0808115
:1011C00084608083E0EBF0E0808181608083EAE7E7
:1011D000F0E0808184608083808182608083808170
:1011E000816080838081806880831092C10008952F
:1011F000833081F028F4813099F08230A1F0089595
:101200008730A9F08830B9F08430D1F48091800023
:101210008F7D03C0809180008F7780938000089538
:1012200084B58F7702C084B58F7D84BD0895809189
:10123000B0008F7703C08091B0008F7D8093B000A5
:101240000895CF93DF9390E0FC01E458FF4F249181
:10125000FC01E057FF4F8491882349F190E0880F0B
:10126000991FFC01E854FF4FA591B49182559F4FFF
:10127000FC01C591D4919FB7611108C0F8948C917D
:10128000209582238C93888182230AC0623051F496
:10129000F8948C91322F309583238C938881822B04
:1012A000888304C0F8948C91822B8C939FBFDF912C
:1012B000CF9108950F931F93CF93DF931F92CDB7D4
:1012C000DEB7282F30E0F901E859FF4F8491F9018A
:1012D000E458FF4F1491F901E057FF4F04910023A8
:1012E000C9F0882321F069830E94F8086981E02F02
:1012F000F0E0EE0FFF1FE255FF4FA591B4919FB7AD
:10130000F8948C91611103C01095812301C0812B49
:101310008C939FBF0F90DF91CF911F910F910895F4
:10132000CF93DF93282F30E0F901E859FF4F8491E4
:10133000F901E458FF4FD491F901E057FF4FC491F0
:10134000CC2391F081110E94F808EC2FF0E0EE0F11
:10135000FF1FEC55FF4FA591B4912C912D2381E0F7
:1013600090E021F480E002C080E090E0DF91CF9136
:101370000895FC01818D228D90E0805C9F4F821B3F
:1013800091098F7399270895FC01918D828D98178B
:1013900031F0828DE80FF11D858D90E008958FEF7B
:1013A0009FEF0895FC01918D828D981761F0828DD9
:1013B000DF01A80FB11D5D968C91928D9F5F9F7389
:1013C000928F90E008958FEF9FEF089586E59BE060
:1013D000892B49F080E090E0892B29F00E94560B80
:1013E00081110C9400000895FC01848DDF01A80F89
:1013F000B11DA35ABF4F2C91848D90E001968F733D
:101400009927848FA689B7892C93A089B1898C915B
:1014100080648C93938D848D981306C00288F38921
:10142000E02D80818F7D80830895CF93DF93EC0141
:10143000888D8823C9F0EA89FB89808185FD05C0F4
:10144000A889B9898C9186FD0FC00FB607FCF5CF2E
:10145000808185FFF2CFA889B9898C9185FFEDCF76
:10146000CE010E94F409E7CFDF91CF910895CF928A
:10147000DF92FF920F931F93CF93DF931F92CDB70D
:10148000DEB76C01DC015B969C915B975C968C915E
:101490005C97981307C05096ED91FC91519780810D
:1014A00085FD32C0F601038D10E00F5F1F4F0F73F3
:1014B0001127F02EF601848DF81211C00FB607FC2B
:1014C000F9CFD6015096ED91FC915197808185FF1F
:1014D000F1CFC60169830E94F4096981EBCF838D46
:1014E000E80FF11DE35AFF4F6083D6015B960C9322
:1014F0005B975296ED91FC91539780818062808337
:1015000081E058968C930DC0D6015696ED91FC91D2
:10151000579760835096ED91FC915197808180643C
:10152000808381E090E00F90DF91CF911F910F9128
:10153000FF90DF90CF900895BF92CF92DF92EF920D
:10154000FF92CF93DF93EC016A017B01B22EE88911
:10155000F98982E08083411581EE580761057105A4
:10156000A1F060E079E08DE390E0A70196010E9490
:10157000B80C2150310941095109569547953795C5
:101580002795211580E1380798F0E889F9891082BC
:1015900060E874E88EE190E0A70196010E94B80C23
:1015A000215031094109510956954795379527959D
:1015B000EC85FD853083EE85FF852083188EEC89D0
:1015C000FD89B082EA89FB89808180618083EA8914
:1015D000FB89808188608083EA89FB8980818068BB
:1015E0008083EA89FB8980818F7D8083DF91CF9121
:1015F000FF90EF90DF90CF90BF9008951F920F92D1
:101600000FB60F9211242F938F939F93EF93FF9315
:10161000E0910204F09103048081E0910804F091CC
:10162000090482FD12C0908180910B048F5F8F733B
:1016300020910C04821751F0E0910B04F0E0EE5081
:10164000FC4F958F80930B0401C08081FF91EF9137
:101650009F918F912F910F900FBE0F901F90189513
:101660001F920F920FB60F9211242F933F934F9317
:101670005F936F937F938F939F93AF93BF93EF93FA
:10168000FF9382EF93E00E94F409FF91EF91BF91E5
:10169000AF919F918F917F916F915F914F913F910A
:1016A0002F910F900FBE0F901F90189582EF93E02F
:1016B0000E94B90921E0892B09F420E0822F0895C6
:1016C0001092F5031092F40388EE93E0A0E0B0E0EE
:1016D0008093F6039093F703A093F803B093F90374
:1016E00080EC91E09093F3038093F20385EC90E01B
:1016F0009093FF038093FE0384EC90E090930104A9
:101700008093000480EC90E09093030480930204A3
:1017100081EC90E0909305048093040482EC90E0C7
:10172000909307048093060486EC90E0909309045C
:101730008093080410920B0410920C0410920D0474
:1017400010920E04089508950E94BD080E94A30BF4
:101750000E94D601C6EED9E00E94F3002097E1F383
:101760000E94E609F9CFCF92DF92EF92FF920F939A
:101770001F93CF93DF936C017A01EB01E60EF71E06
:1017800000E010E0CE15DF0561F06991D601ED9122
:10179000FC910190F081E02DC6010995080F191FF9
:1017A000F1CFC801DF91CF911F910F91FF90EF9082
:1017B000DF90CF9008956115710581F0DB010D90E8
:1017C0000020E9F7AD0141505109461B570BDC01E0
:1017D000ED91FC910280F381E02D099480E090E08E
:1017E00008950C94DB0BDC01ED91FC910190F081EC
:1017F000E02D09940F931F93CF93DF93EC016DE0DD
:101800000E94F30B8C016AE0CE010E94F30B800F63
:10181000911FDF91CF911F910F9108950F931F9307
:10182000CF93DF93EC010E94DB0B8C01CE010E9471
:10183000FA0B800F911FDF91CF911F910F910895A7
:101840008F929F92AF92BF92CF92DF92EF92FF92D0
:101850000F931F93CF93DF93CDB7DEB7A1970FB64A
:10186000F894DEBF0FBECDBF7C01C42EE52FCB01A7
:10187000D22E19A221E02D1510F02AE0D22E8E01D1
:101880000F5D1F4F8D2C912CA12CB12C6C2D7E2F18
:10189000A50194010E94B80C8C2DD29E80191124B0
:1018A000015011098A3014F4805D01C0895CF8018F
:1018B0008083211531054105510521F0C22EE32F0A
:1018C000CA01E4CFB801C7010E94DB0BA1960FB695
:1018D000F894DEBF0FBECDBFDF91CF911F910F9166
:1018E000FF90EF90DF90CF90BF90AF909F908F9040
:1018F00008952115310541F4DC01ED91FC91019031
:10190000F081E02D642F09940C94200C9A01462F4D
:1019100050E060E070E00C94790C0F931F93CF932C
:10192000DF93EC019A01AB0160E070E00E94790C5A
:101930008C01CE010E94FA0B800F911FDF91CF9195
:101940001F910F910895089597FB072E16F40094A8
:1019500007D077FD09D00E94E00C07FC05D03EF4CB
:10196000909581959F4F0895709561957F4F08954B
:10197000A1E21A2EAA1BBB1BFD010DC0AA1FBB1F93
:10198000EE1FFF1FA217B307E407F50720F0A21B05
:10199000B30BE40BF50B661F771F881F991F1A9472
:1019A00069F760957095809590959B01AC01BD019C
:1019B000CF010895EE0FFF1F0590F491E02D0994DB
:1019C000AA1BBB1B51E107C0AA1FBB1FA617B70765
:1019D00010F0A61BB70B881F991F5A95A9F7809581
:0C19E0009095BC01CD010895F894FFCF54
:1019EC002030004352433136202868657829203A4C
:1019FC0020004352433136202862696E29203A2058
:101A0C00005549442053697A653A20004361726459
:101A1C002055494428686578293A004D465243358B
:101A2C00323220536F66747761726520566572731B
:101A3C00696F6E3A203078005741524E494E473A02
:101A4C0020436F6D6D756E69636174696F6E20668E
:101A5C0061696C7572652C20697320746865204D02
:101A6C004652433532322070726F7065726C792039
:101A7C00636F6E6E65637465643F0050726F67725E
:101A8C00616D6D3A20524649442D5338382D4C69BE
:101A9C006768745F4352432D5630310000000000DC
:0C1AAC00370AB30BB909D209C409150AA6
:00000001FF
